:100000000C945B000C9463040C9490040C94830097
:100010000C9483000C9483000C9483000C94830054
:100020000C9483000C9483000C9483000C94830044
:100030000C9483000C9483000C9483000C94830034
:100040000C94BD040C9483000C94E1060C94830082
:100050000C9483000C9483000C9483000C94830014
:100060000C9483000C948300000024272A000025B0
:10007000282B000023262904040404040404040299
:100080000202020202030303030303010204081035
:100090002040800102040810200102040810200002
:1000A0000000070002010000030406000000000039
:1000B000000000003A0311241FBECFEFD8E0DEBFDE
:1000C000CDBF11E0A0E0B1E0E4E1FFE002C00590A7
:1000D0000D92AA33B107D9F711E0AAE3B1E001C04C
:1000E0001D92AD3DB107E1F710E0C6EBD0E004C0D2
:1000F0002297FE010E948407C43BD107C9F70E94E2
:1001000033030C9488070C94000040E855E260E04B
:1001100070E087E491E00E944B0364E670E080E0C9
:1001200090E00E942D0561E080911B010E9407066E
:1001300061E080911D010E94070661E080911F012E
:100140000E94070660E08EE00E94070660E08FE0F4
:100150000E94070660E080E10E94070660E081E1FE
:100160000E94070661E08EE00E94250661E08FE0B4
:100170000E94250661E080E10E94250661E081E1A0
:100180000E94250680913A010E949105815092407B
:100190003CF080E190E090933D0180933C0104C0ED
:1001A00010923D0110923C01809121010E94910525
:1001B000815092403CF080E290E090933F01809328
:1001C0003E0104C010923F0110923E018091230134
:1001D0000E949105815092403CF080E490E0909321
:1001E00041018093400104C01092410110924001EE
:1001F000809125010E949105815092403CF080E859
:1002000090E0909343018093420104C01092430117
:100210001092420180913E0190913F0120913C015A
:1002200030913D01820F931F209140013091410197
:10023000820F931F2091420130914301820F931F3F
:10024000909346018093450160E071E087E491E07E
:100250000E945003609145017091460187E491E04E
:100260000E943E04089560E080912B010E942506C3
:1002700060E080912D010E94250660E070E0809191
:1002800027010E94AF0560E080912F010E942506A2
:1002900060E0809131010E94250660E070E080916D
:1002A00029010E94AF0508950F931F93CF93DF9309
:1002B0008C010E94330164E670E080E090E00E94CF
:1002C0002D0560E080912F010E94250661E080915C
:1002D00031010E94250660E080912B010E942506D5
:1002E00061E080912D010E942506C0E4D0E011C09C
:1002F000BE01809127010E94AF05BE0180912901B6
:100300000E94AF0564E670E080E090E00E942D0559
:100310002A960C171D0764F7B801809129010E94E5
:10032000AF05B801809127010E94AF05DF91CF9101
:100330001F910F9108950F931F93CF93DF938C011B
:100340000E94330164E670E080E090E00E942D0599
:1003500061E080912F010E94250660E080913101CB
:100360000E94250661E080912B010E94250660E035
:1003700080912D010E942506C0E4D0E011C0BE018D
:10038000809127010E94AF05BE01809129010E9442
:10039000AF0564E670E080E090E00E942D052A96AB
:1003A0000C171D0764F7B801809129010E94AF0561
:1003B000B801809127010E94AF05DF91CF911F9175
:1003C0000F9108950F931F93CF93DF938C010E9499
:1003D000330164E670E080E090E00E942D0561E06A
:1003E00080912F010E94250660E0809131010E94DA
:1003F000250660E080912B010E94250660E0809137
:100400002D010E94250660E070E0809127010E9486
:10041000AF05C0E4D0E00CC0BE01809129010E946C
:10042000AF0564E670E080E090E00E942D052A961A
:100430000C171D078CF7B801809129010E94AF05A8
:10044000DF91CF911F910F9108950F931F93CF9339
:10045000DF938C010E94330164E670E080E090E05D
:100460000E942D0561E080912B010E94250660E02D
:1004700080912D010E94250660E080912F010E944D
:10048000250660E0809131010E94250660E070E061
:10049000809129010E94AF05C0E4D0E00CC0BE01EC
:1004A000809127010E94AF0564E670E080E090E053
:1004B0000E942D052A960C171D078CF7B801809114
:1004C00027010E94AF05DF91CF911F910F910895F1
:1004D00061E080911B010E94250668EE73E080E0D8
:1004E00090E00E942D0560E080911B010E9425068E
:1004F00068EE73E080E090E00E942D0587E491E0D3
:100500000E944803882309F4ADC087E491E00E946B
:1005100045038093440190E0A0E0B0E020E030E0AB
:10052000AC01BD0187E491E00E944E04409144017A
:10053000842F90E0807F907020914501309146019A
:100540008217930709F08EC050E060E070E020E071
:1005500030E087E491E00E944E048091440190E0F5
:100560008F7090708730910509F453C088309105E1
:10057000B4F48330910509F43CC0843091054CF407
:100580008130910551F18230910564F5892B01F19B
:10059000089585309105B9F10697C4F531C08B30C7
:1005A000910509F448C08C30910534F489309105E7
:1005B000E1F10A97ECF536C08D30910509F447C09A
:1005C0008D3091050CF440C00E9709F04BC045C02A
:1005D0008FEF90E00E94540108958FEF90E00E9409
:1005E0009B0108958FEF90E00E94250280E090E04B
:1005F00028C08FEF90E00E94E20180E090E00FC001
:1006000084EB90E008C080E890E005C080E590E0D1
:1006100002C080E490E00E94E2018FEF90E00E942F
:100620002502089584EB90E008C080E890E005C0C2
:1006300080E590E002C080E490E00E9425028FEF08
:1006400090E00E94E20108950E943301089561E064
:1006500080911F010E942506089560E080911F018E
:100660000E94250608950E9457050E9485000E9459
:100670006802FDCF88E391E09093480180934701A1
:100680000895862F0E94A90608950E94C206089523
:100690000E94B1060895CB01BA010E947006089528
:1006A0000F931F93CF93DF938C01EB0109C0219629
:1006B000D801ED91FC910190F081E02DC8010995E0
:1006C00068816623A1F7DF91CF911F910F91089563
:1006D0000F931F938C01DC01ED91FC910190F0814F
:1006E000E02D6DE00995D801ED91FC910190F0812C
:1006F000E02D6AE0C80109951F910F9108952F928E
:100700003F924F925F926F927F928F929F92AF92A1
:10071000BF92CF92DF92EF92FF920F931F93DF93DE
:10072000CF93CDB7DEB7A0970FB6F894DEBF0FBE5C
:10073000CDBF1C016A017B014115510561057105A1
:1007400049F4DC01ED91FC910190F081E02D60E332
:10075000099554C0882499245401422E55246624B6
:10076000772401E010E00C0F1D1F080D191DC701B3
:10077000B601A30192010E943107F8016083089439
:10078000811C911CA11CB11CC701B601A3019201DF
:100790000E943107C901DA016C017D01C114D10445
:1007A000E104F104F1F681E0E82EF12CEC0EFD1EDF
:1007B000E80CF91C3E010894611C711CD501C401B0
:1007C0000197A109B1096C01C818D90814C0F60134
:1007D000EE0DFF1D60816A3010F4605D01C0695C40
:1007E000D101ED91FC910190F081E02DC1010995BD
:1007F0000894E108F1086E147F0449F7A0960FB63B
:10080000F894DEBF0FBECDBFCF91DF911F910F9146
:10081000FF90EF90DF90CF90BF90AF909F908F9020
:100820007F906F905F904F903F902F900895EF9240
:10083000FF920F931F93CF93DF93EC017A018B010B
:1008400077FF0FC0E881F9810190F081E02D6DE222
:10085000099510950095F094E094E11CF11C011DA0
:10086000111D2AE0B801A701CE010E947F03DF918C
:10087000CF911F910F91FF90EF9008950F931F93C9
:100880008C01AB01662757FD6095762F0E941704F7
:10089000C8010E9468031F910F910895DC01211582
:1008A000310541F4ED91FC910190F081E02D642F30
:1008B000099508952A30310519F40E941704089506
:1008C0000E947F0308951F920F920FB60F9211247A
:1008D0002F933F934F935F936F937F938F939F9348
:1008E000AF93BF93EF93FF938091490190914A0199
:1008F000892B29F0E0914901F0914A010995FF9176
:10090000EF91BF91AF919F918F917F916F915F9187
:100910004F913F912F910F900FBE0F901F90189500
:100920001F920F920FB60F9211242F933F934F9364
:100930005F936F937F938F939F93AF93BF93EF9347
:10094000FF9380914B0190914C01892B29F0E0910C
:100950004B01F0914C010995FF91EF91BF91AF913F
:100960009F918F917F916F915F914F913F912F91C7
:100970000F900FBE0F901F9018951F920F920FB6F9
:100980000F9211242F938F939F93AF93BF938091D6
:100990004D0190914E01A0914F01B09150010196EF
:1009A000A11DB11D80934D0190934E01A0934F0165
:1009B000B09350018091510190915201A091530147
:1009C000B09154018050904CAF4FBF4F8093510174
:1009D00090935201A0935301B093540127C080918A
:1009E000510190915201A0915301B091540180584E
:1009F0009E43A040B0408093510190935201A09338
:100A00005301B09354018091550190915601A091EA
:100A10005701B09158010196A11DB11D8093550158
:100A200090935601A0935701B093580180915101C2
:100A300090915201A0915301B091540181589E436D
:100A4000A040B04060F6BF91AF919F918F912F91E0
:100A50000F900FBE0F901F901895EF92FF920F937B
:100A60001F937B018C018FB7F894409155015091F1
:100A7000560160915701709158018FBF2FB7F894BC
:100A80008091550190915601A0915701B091580164
:100A90002FBF841B950BA60BB70BE816F9060A07A8
:100AA0001B0760F71F910F91FF90EF9008957894C6
:100AB00084B5826084BD84B5816084BD85B5826063
:100AC00085BD85B5816085BDEEE6F0E08081816001
:100AD0008083E1E8F0E080818260808380818160B2
:100AE0008083E0E8F0E0808181608083E1EBF0E0EA
:100AF000808184608083E0EBF0E08081816080838E
:100B0000EAE7F0E080818460808380818260808376
:100B10008081816080838081806880831092C100A1
:100B200008958F70909133019295990F990F907C51
:100B3000982B90937C0080917A00806480937A0057
:100B400080917A0086FDFCCF209178004091790059
:100B5000942F80E030E0282B392BC90108951F9392
:100B6000CF93DF93182FEB0161E00E940706E12F7E
:100B7000F0E0E156FF4F8491833051F48091800082
:100B8000806880938000D0938900C09388003BC028
:100B9000843051F480918000806280938000D093F3
:100BA0008B00C0938A002FC0813039F4209729F13F
:100BB00084B5806884BDC7BD26C0823039F42097D3
:100BC000E1F084B5806284BDC8BD1DC0863041F4AB
:100BD0008091B00080688093B000C093B30013C0D0
:100BE000873041F48091B00080628093B000C09360
:100BF000B40009C0C038D10514F460E001C061E060
:100C0000812F0E942506DF91CF911F910895282FF3
:100C100030E0C90185579F4FFC01949129583F4FFF
:100C2000F9018491882381F0E82FF0E0E859FF4F23
:100C3000E491F0E0662329F48081909589238083F4
:100C400008958081892B80830895482F50E0CA0140
:100C500081569F4FFC012491CA0185579F4FFC018B
:100C6000949149585F4FFA0134913323C1F1222303
:100C700031F1233021F4809180008F7705C024303A
:100C800031F4809180008F7D8093800018C02130E6
:100C900019F484B58F7704C0223021F484B58F7D98
:100CA00084BD0DC0263021F48091B0008F7705C03F
:100CB000273029F48091B0008F7D8093B000E32F1E
:100CC000F0E0E359FF4FE491F0E0662329F48081DE
:100CD00090958923808308958081892B808308954E
:100CE000EF92FF920F931F937B018C0122E030E083
:100CF00040E050E00E945307205C3D4B404F5F4F67
:100D0000CA01B901A80197010E945307C901DA017C
:100D10000197A109B109292F3A2F4B2F552747FDDC
:100D20005A950196A11DB11D2093C5008150809355
:100D3000C400E1ECF0E08081806180838081886084
:100D400080838081806880831F910F91FF90EF9056
:100D50000895982F8091C00085FFFCCF9093C60026
:100D600008958091590190915A0180589F4F209188
:100D70005B0130915C01821B930B60E870E00E9484
:100D80001E07089540915B0150915C0180915901CB
:100D900090915A018417950719F42FEF3FEF0FC078
:100DA000FA01E35AFE4F2081CA01019660E870E023
:100DB0000E941E0790935C0180935B0130E0C901A3
:100DC00008951F920F920FB60F9211242F933F9305
:100DD0004F935F936F937F938F939F93AF93BF9343
:100DE000EF93FF934091C600E0915901F0915A01B1
:100DF000CF01019660E870E00E941E079C0180917F
:100E00005B0190915C012817390739F0E35AFE4FD6
:100E1000408330935A0120935901FF91EF91BF9184
:100E2000AF919F918F917F916F915F914F913F9182
:100E30002F910F900FBE0F901F90189597FB092EC2
:100E400007260AD077FD04D049D006D000201AF436
:100E5000709561957F4F0895F6F7909581959F4F16
:100E60000895A1E21A2EAA1BBB1BFD010DC0AA1FEB
:100E7000BB1FEE1FFF1FA217B307E407F50720F003
:100E8000A21BB30BE40BF50B661F771F881F991F7E
:100E90001A9469F760957095809590959B01AC01C7
:100EA000BD01CF01089597FB092E05260ED057FDF1
:100EB00004D0D7DF0AD0001C38F450954095309507
:100EC00021953F4F4F4F5F4F0895F6F790958095CE
:100ED000709561957F4F8F4F9F4F0895AA1BBB1B45
:100EE00051E107C0AA1FBB1FA617B70710F0A61B2A
:100EF000B70B881F991F5A95A9F780959095BC014B
:100F0000CD010895EE0FFF1F0590F491E02D099497
:040F1000F894FFCF83
:100F1400486F6C612C20736F7920656C20726F624E
:100F24006F74206E756D65726F2000060008000BEB
:100F34000001000200030009000A0002000300058A
:0A0F4400000400010000000041035A
:00000001FF
